:10000000831602309F008901860183120730890020
:10001000FF3086005620003086002130A6002608DA
:100020002420A500251C20282228091100000915DC
:10003000A60B0F28891400000910000009141F28BE
:10004000891015288914152882070000003400340F
:1000500001340034003401340134003400340034FD
:1000600001340034003401340034013401340034EC
:1000700001340034003400340034003400340034DF
:100080000134013400340034013401340134A5302A
:10009000A00000000000A00B4B2808006330A10066
:1000A000000000004720A10B522808006330A20086
:1000B0006230A3000330A40000004E20A20B5D2894
:0C00C0004720A30B6028A40B6328080055
:00000001FF
